:1000000000308A00812800000A108A100A11820735
:10001000733475346D3420346F3466342034703466
:10002000653461346B347334203470346534723425
:100030002034313473343A340A340D3400342530EA
:10004000840083130008031933280130F800F701F6
:10005000F70B2828F80B27284A30F700F70B2E2833
:100060003128800B252800342708F80126020318C0
:100070003C282608F7004828F7010830A800A60DFC
:10008000F70D270877020318F700F80DA80B3F2893
:10009000003478082408A6006430A70034207708CC
:1000A000A40078083030031D5C28A51C6428A5191D
:1000B0006428251A20305F28A51125122514F80779
:1000C00078080C1E612899002408A6000A30A700B1
:1000D00034207708A40078083030031D7528A5194E
:1000E0007A28251C7A28251A2030F80778080C1E53
:1000F000772899003030A40724080C1E7D28990029
:100100004C29840183131F3083051930831699000D
:10011000A630980090308312980083161F149F1405
:100120001F159F1107309C00FF308312A000A30110
:1001300083161F149F141F159F1183121F108316FF
:10014000091283129412A0122008831687008312CA
:1001500020162008831687008312A011200883161A
:100160008700013083129400003083169400010848
:10017000C73928388100B730831290000030F8006A
:1001800004389200FF308316920083122011200859
:1001900083168700831207110C309700A0102008E7
:1001A00083168700831287100C309D004230950023
:1001B0001708CF391038970042309B001D08CF39FF
:1001C00010389D00073083169C0005080330F700A7
:1001D000F70BE8281C0883120D1383169D01831268
:1001E000A3012308043C031C32290108A1002108B3
:1001F000210203192929A10A0F08FA000E08F700A5
:100200000F087A02031DFC287708A200A20AA2099F
:100210000319292920122008831687008312071248
:10022000A012200883168700831287160230A400CC
:100230009630A5001F20A40B182920122008831631
:10024000870083120716A0122008831687008312E6
:1002500087120230A400FA30A5001F20A40B2B291E
:10026000A30AF1280A300C1E332999000D300C1E08
:1002700037299900A40124080420A40AF70077086C
:100280000C1E4029990016302402031D3B29210829
:0E029000A4001B30A50049288101F02863005E
:02400E0039393E
:00000001FF
